:020000040000fa
:080000000002040000000000f2
:020000040000fa
:040008009a03000057
:020000040000fa
:04000c00b403000039
:020000040000fa
:040010006603000083
:020000040000fa
:04001400ce03000017
:020000040000fa
:04001800e8030000f9
:020000040000fa
:04001c0032030000ab
:020000040000fa
:040020008003000059
:020000040000fa
:040024004c03000089
:020000040000fa
:040028003c04000094
:020000040000fa
:04002c003c04000090
:020000040000fa
:040030003c0400008c
:020000040000fa
:040034003c04000088
:020000040000fa
:040038003c04000084
:020000040000fa
:04003c003c04000080
:020000040000fa
:040040003c0400007c
:020000040000fa
:040044003c04000078
:020000040000fa
:040048003c04000074
:020000040000fa
:04004c003c04000070
:020000040000fa
:040050003c0400006c
:020000040000fa
:040054003c04000068
:020000040000fa
:040058003c04000064
:020000040000fa
:04005c003c04000060
:020000040000fa
:040060003c0400005c
:020000040000fa
:040064003c04000058
:020000040000fa
:040068003c04000054
:020000040000fa
:04006c003c04000050
:020000040000fa
:040070003c0400004c
:020000040000fa
:040074003c04000048
:020000040000fa
:040078003c04000044
:020000040000fa
:04007c003c04000040
:020000040000fa
:040080003c0400003c
:020000040000fa
:040084003c04000038
:020000040000fa
:040088003c04000034
:020000040000fa
:04008c003c04000030
:020000040000fa
:040090003c0400002c
:020000040000fa
:040094003c04000028
:020000040000fa
:040098003c04000024
:020000040000fa
:04009c003c04000020
:020000040000fa
:0400a0003c0400001c
:020000040000fa
:0400a4003c04000018
:020000040000fa
:0400a8003c04000014
:020000040000fa
:0400ac003c04000010
:020000040000fa
:0400b0003c0400000c
:020000040000fa
:0400b4003c04000008
:020000040000fa
:0400b8003c04000004
:020000040000fa
:0400bc003c04000000
:020000040000fa
:0400c0003c040000fc
:020000040000fa
:0400c4003c040000f8
:020000040000fa
:0400c8003c040000f4
:020000040000fa
:0400cc003c040000f0
:020000040000fa
:0400d0003c040000ec
:020000040000fa
:0400d4003c040000e8
:020000040000fa
:0400d8003c040000e4
:020000040000fa
:0400dc003c040000e0
:020000040000fa
:0400e0003c040000dc
:020000040000fa
:0400e4003c040000d8
:020000040000fa
:0400e8003c040000d4
:020000040000fa
:0400ec003c040000d0
:020000040000fa
:0400f0003c040000cc
:020000040000fa
:0400f4003c040000c8
:020000040000fa
:0400f8003c040000c4
:020000040000fa
:0400fc003c040000c0
:020000040000fa
:040100003c040000bb
:020000040000fa
:040104003c040000b7
:020000040000fa
:040108003c040000b3
:020000040000fa
:04010c003c040000af
:020000040000fa
:040110003c040000ab
:020000040000fa
:040114003c040000a7
:020000040000fa
:040118003c040000a3
:020000040000fa
:04011c003c0400009f
:020000040000fa
:040120003c0400009b
:020000040000fa
:040124003c04000097
:020000040000fa
:040128003c04000093
:020000040000fa
:04012c003c0400008f
:020000040000fa
:040130003c0400008b
:020000040000fa
:040134003c04000087
:020000040000fa
:040138003c04000083
:020000040000fa
:04013c003c0400007f
:020000040000fa
:040140003c0400007b
:020000040000fa
:040144003c04000077
:020000040000fa
:040148003c04000073
:020000040000fa
:04014c003c0400006f
:020000040000fa
:040150003c0400006b
:020000040000fa
:040154003c04000067
:020000040000fa
:040158003c04000063
:020000040000fa
:04015c003c0400005f
:020000040000fa
:040160003c0400005b
:020000040000fa
:040164003c04000057
:020000040000fa
:040168003c04000053
:020000040000fa
:04016c003c0400004f
:020000040000fa
:040170003c0400004b
:020000040000fa
:040174003c04000047
:020000040000fa
:040178003c04000043
:020000040000fa
:04017c003c0400003f
:020000040000fa
:040180003c0400003b
:020000040000fa
:040184003c04000037
:020000040000fa
:040188003c04000033
:020000040000fa
:04018c003c0400002f
:020000040000fa
:040190003c0400002b
:020000040000fa
:040194000204000061
:020000040000fa
:040198003c04000023
:020000040000fa
:04019c003c0400001f
:020000040000fa
:0401a0003c0400001b
:020000040000fa
:0401a4003c04000017
:020000040000fa
:0401a8003c04000013
:020000040000fa
:0401ac003c0400000f
:020000040000fa
:0401b0003c0400000b
:020000040000fa
:0401b4003c04000007
:020000040000fa
:0401b8003c04000003
:020000040000fa
:0401bc003c040000ff
:020000040000fa
:0401c0003c040000fb
:020000040000fa
:0401c4003c040000f7
:020000040000fa
:0401c8003c040000f3
:020000040000fa
:0401cc003c040000ef
:020000040000fa
:0401d0003c040000eb
:020000040000fa
:0401d4003c040000e7
:020000040000fa
:0401d8003c040000e3
:020000040000fa
:0401dc003c040000df
:020000040000fa
:0401e0003c040000db
:020000040000fa
:0401e4003c040000d7
:020000040000fa
:0401e8003c040000d3
:020000040000fa
:0401ec003c040000cf
:020000040000fa
:0401f0003c040000cb
:020000040000fa
:0401f4003c040000c7
:020000040000fa
:0401f8003c040000c3
:020000040000fa
:0401fc003c040000bf
:020000040000fa
:040200003c040000ba
:020000040000fa
:040204003c040000b6
:020000040000fa
:040208003c040000b2
:020000040000fa
:04020c003c040000ae
:020000040000fa
:040210003c040000aa
:020000040000fa
:040214003c040000a6
:020000040000fa
:040218003c040000a2
:020000040000fa
:04021c003c0400009e
:020000040000fa
:040220003c0400009a
:020000040000fa
:040224003c04000096
:020000040000fa
:040228003c04000092
:020000040000fa
:04022c003c0400008e
:020000040000fa
:040230003c0400008a
:020000040000fa
:040234003c04000086
:020000040000fa
:040238003c04000082
:020000040000fa
:04023c003c0400007e
:020000040000fa
:040240003c0400007a
:020000040000fa
:040244003c04000076
:020000040000fa
:040248003c04000072
:020000040000fa
:04024c003c0400006e
:020000040000fa
:040250003c0400006a
:020000040000fa
:040254003c04000066
:020000040000fa
:040258003c04000062
:020000040000fa
:04025c003c0400005e
:020000040000fa
:040260003c0400005a
:020000040000fa
:040264003c04000056
:020000040000fa
:040268003c04000052
:020000040000fa
:04026c003c0400004e
:020000040000fa
:040270003c0400004a
:020000040000fa
:040274003c04000046
:020000040000fa
:040278003c04000042
:020000040000fa
:04027c003c0400003e
:020000040000fa
:040280003c0400003a
:020000040000fa
:040284003c04000036
:020000040000fa
:040288003c04000032
:020000040000fa
:04028c003c0400002e
:020000040000fa
:040290003c0400002a
:020000040000fa
:040294003c04000026
:020000040000fa
:040298003c04000022
:020000040000fa
:04029c003c0400001e
:020000040000fa
:0402a0003c0400001a
:020000040000fa
:0402a4003c04000016
:020000040000fa
:0402a8003c04000012
:020000040000fa
:0402ac003c0400000e
:020000040000fa
:0402b0003c0400000a
:020000040000fa
:0402b4003c04000006
:020000040000fa
:0402b8003c04000002
:020000040000fa
:0402bc003c040000fe
:020000040000fa
:0402c0003c040000fa
:020000040000fa
:0402c4003c040000f6
:020000040000fa
:0402c8003c040000f2
:020000040000fa
:0402cc003c040000ee
:020000040000fa
:0402d0003c040000ea
:020000040000fa
:0402d4003c040000e6
:020000040000fa
:0402d8003c040000e2
:020000040000fa
:0402dc003c040000de
:020000040000fa
:0402e0003c040000da
:020000040000fa
:0402e4003c040000d6
:020000040000fa
:0402e8003c040000d2
:020000040000fa
:0402ec003c040000ce
:020000040000fa
:0402f0003c040000ca
:020000040000fa
:0402f4003c040000c6
:020000040000fa
:0402f8003c040000c2
:020000040000fa
:0402fc003c040000be
:020000040000fa
:040300003c040000b9
:020000040000fa
:040304003c040000b5
:020000040000fa
:040308003c040000b1
:020000040000fa
:04030c003c040000ad
:020000040000fa
:040310003c040000a9
:020000040000fa
:040314003c040000a5
:020000040000fa
:040318003c040000a1
:020000040000fa
:04031c003c0400009d
:020000040000fa
:040320003c04000099
:020000040000fa
:040324003c04000095
:020000040000fa
:100400006f3921002efd22000e018800000000003f
:10041000000020000000e000020032000001200087
:100420002002880014000700150107000000e0000a
:1004300003003a0080df21000100200002003700a5
:100440000000200001002000810f70000100320038
:100450000f000700000020000000e0000200320052
:100460000000020000000000a223020000000000c3
:100470000040da000000fe00200020000000e00044
:1004800002003200100020009001880000000600e9
:10049000a1028800800478000000eb001f003700f4
:1004a000e284440054a0b4009905ba00e2844400f8
:1004b00054a0b4009906ba00e284440054a0b400e9
:1004c0000006eb00476fde00fd07b200ae018800ba
:1004d000636ce10003003a000ad801000000eb0061
:1004e0000e003700606ce10008003a00004deb00a0
:1004f0000a05e800020039003420ec000af0a000f0
:100500008b05e900f9ff3e00040037006168e10057
:10051000010032000086eb000b00070019c7ba008b
:100520001905ba000e04e00003003a000a00e000da
:10053000dbff3a0000000600fe07b200ae028800b2
:100540008a047800f5ff37000cd0a300e20f4d00bd
:100550001c00390089027800354dba000a05e80010
:10056000020039003420ec000af0a0008b05e900fd
:100570000f003200254dba000a05e80002003900dc
:100580003420ec000af0a0008b05e90008003200de
:100590000c00e0000600320015cdba000a05e800a4
:1005a000020039003420ec000af0a0008b05e900bd
:1005b0008984e80054a0b4000b00e000e2ff3a0098
:1005c000000006009902ba00055d78008b05e9007d
:1005d000f7ff3200c82ade00055d78008b05e900d0
:1005e000f3ff32000c00e000f1ff320019ddba0029
:1005f000eeff3700000000000000000000000000d7
:1006000000000000000000000000000000000000ea
:1006100000000000000000000000000000000000da
:1006200000000000000000000000000000000000ca
:1006300000000000000000000000000000000000ba
:1006400000000000000000000000000000000000aa
:10065000000000000000000000000000000000009a
:10066000000000003600f800809fbe00829fbe00a0
:10067000849fbe00869fbe0000082000491307002b
:100680004f03be004f02be004f01be004f00be0030
:100690003600f900004006003600f800809fbe00da
:1006a000829fbe00849fbe00869fbe00000820007f
:1006b0003c1307004f03be004f02be004f01be00b7
:1006c0004f00be003600f900004006003600f8007a
:1006d000809fbe00829fbe00849fbe00869fbe009a
:1006e000000420002f1307004f03be004f02be007e
:1006f0004f01be004f00be003600f900004006006a
:100700003600f800809fbe00829fbe00849fbe001e
:10071000869fbe0000022000221307004f03be0088
:100720004f02be004f01be004f00be003600f90070
:10073000004006003600f800809fbe00829fbe0089
:10074000849fbe00869fbe00100020001513070086
:100750004f03be004f02be004f01be004f00be005f
:100760003600f900004006003600f800809fbe0009
:10077000829fbe00849fbe00869fbe002000200096
:10078000081307004f03be004f02be004f01be001a
:100790004f00be003600f900004006003600f800a9
:1007a000809fbe00829fbe00849fbe00869fbe00c9
:1007b00040002000fb1207004f03be004f02be00a6
:1007c0004f01be004f00be003600f9000040060099
:1007d0003600f800809fbe00829fbe00849fbe004e
:1007e000869fbe0080002000ee1207004f03be006f
:1007f0004f02be004f01be004f00be003600f900a0
:10080000004006003600f8003200f8003400f8001e
:1008100010002000a0018800100020009001880036
:1008200023cea800800921001010a000a18c800018
:10083000708c800001000100418d8000108d8000cf
:1008400001000100e18d8000b08d800001000100f9
:100850000000000000000000000000000000000098
:100860000b68a90023cea9003400f9003200f9007a
:100870003600f900004006000040da000000fe00eb
:04088000000005006f
:020000040000fa
:100884001000fa00889fbe000004780010002000c9
:10089400e0b79f000000eb00f0b79f006000b800d5
:1008a40080bf9f0091bf9f00a0bf9f00b1bf9f006a
:1008b400c0bf9f00d1bf9f001800e00002003d00b0
:1008c4001838a30014003a00980078006180600092
:1008d4000004e0000d003a000000eb001004980052
:1008e400180090008000eb00e90f5000e08f5800e2
:1008f400100036000000eb00100498006fb0970061
:100904004f04be000080fa00000006001000200022
:1009140010049800f2ff37001878a300f0ff3200ab
:1009240098007800618060000004e000f7ff3a005e
:10093400e9ff3700000601002401370001013700f8
:10094400e7003700d40037005f003700410037006c
:10095400360037001e003700010037002d01370034
:10096400b810900068b09000808f50007802320078
:100974001880a000b810900068b09000808f5000dc
:1009840089013900b810900068b09000808f500041
:10099400daff360068b090009810900000804000a4
:1009a40060b49800e8b0900038109000808f500038
:1009b400d2ff36003810900060b498006fb09700f2
:1009c4004f04be000080fa0000000600cfff37008d
:1009d4001880a00068009000f80090000001e80072
:1009e40062049800810f5000c4ff3600800020008c
:1009f40010049800780090000000e800600498005b
:100a040028e091000004e000bcff3200200e20002a
:100a140008004000091107006fb097004f04be00a2
:100a24000080fa0000000600b8ff3700281090008c
:100a3400e20f50009301320038b89000a8b890003b
:100a440010219000112098007000200010049800dc
:100a5400aaff37001880a00038b89000104090001a
:100a64000078a300a20132000810900098109000b2
:100a740000804000001498008810900068b0900036
:100a8400808f50009dff360068b0900000149800dd
:100a940038b89000c10e20008880400010119000ea
:100aa40011109800281090000000e000e6ff3200ca
:100ab40028109000e20f500090ff3a0060002000e0
:100ac400100498008dff37001880a0000000eb0090
:100ad40000149800e0032000400c980038b89000ff
:100ae400010220008880400010119000111098002d
:100af400281890000014980028109000e20f50006d
:100b0400910132009818900058209000808f500076
:100b1400d4003200a818900078289000808f5000ec
:100b2400d0003200d828900028199000782890002e
:100b3400000051000100b80080bf9f0091bf9f00da
:100b44000fb897009fb897006829900070011100b2
:100b54000201e900030033008100d1000080d300ca
:100b6400fbff370080bf9f0091bf9f00b82090001b
:100b74001819900058209000000051000100b8009e
:100b8400a0bf9f00b1bf9f002fb89700bfb89700c8
:100b940048219000700111000201e90003003300b4
:100ba4008100d1000080d300fbff3700a0bf9f006d
:100bb400b1bf9f00389190000fb897009fb897007d
:100bc4000200b800c0bf9f00d1bf9f002fb997009b
:100bd400bfb997004fba9700dfba97000500090024
:100be40042aad8008000eb00c0bf9f00d1bf9f0085
:100bf400281090000000e000a1003a0018b990000d
:100c04004fb89700dfb89700cf91de00800f5100f6
:100c1400818f5900c201360018b89000cf80de00e1
:100c2400c0bf9f00d1bf9f00f8b990004fba970092
:100c3400dfba970038b89000040178008000eb0018
:100c44000300010038b89000a05090008180fb00a0
:100c5400305090004800dd00008070004fb99700cc
:100c6400dfb997000208780038b89000a0589000c7
:100c74008180fb00305890004800dd000080700047
:100c84004fb99700dfb997000208780050002000a0
:100c94001004980019ff37001880a0002800900065
:100ca400b80090000001e80022049800810f500071
:100cb40012ff3600380090000000e800200498007d
:100cc400400020001848a3000bff3a006fb09700c3
:100cd4004f04be000080fa00000006000bff37003e
:100ce4001880a1001800e00003003d0018e8a300ec
:100cf4000100320018d0a00008d891000004e000e0
:100d040008013a001800e000fcfe3d0018d8a300da
:100d1400fafe32001818a300f8fe32001828a300c7
:100d2400f6fe32001878a300f4fe3a001848a30037
:100d3400f2fe320018d0a100300020001004980008
:100d4400eefe37001880a00008007800cd0e0700e2
:100d5400efb0970001006000e0b79f00b8b89000c2
:100d6400114090000074a10090409800d8b8900001
:100d740038b890000100010038b89000205190006c
:100d84000281fb00b0509000c808dd0081007100b2
:100d940038b8900000c190000281fb0010c09000a0
:100da4004800dd0082087000e0858000e20f5000fa
:100db400ec00320028e091000004e00089003a00d1
:100dc4002000200010049800ccfe37001880a000fa
:100dd4000000eb0020049800600498001830a10083
:100de4001810a1001898a3006d0032001840a1004b
:100df40028e091000004e00003003200200e2000ef
:100e0400080040003510070010002000100498006e
:100e1400bafe370008007800f80c0700efb097001e
:100e240001006000e0b79f00b8b890001140900046
:100e34000074a1009040980028109000e20f500028
:100e44006d003200380090000000e8002004980093
:100e5400780090000000e800600498001000200072
:100e6400eaff3700689090008000eb00c0bf9f004d
:100e7400d1bf9f00281090000000e0005fff320007
:100e840028109000e20f500080ff3a000000eb00b1
:100e9400f0b79f0010868000ffb09700808f50004d
:100ea4007aff31007fb097007400b9006010b00081
:100eb400680178004fb89700dfb89700cf91de0043
:100ec400800f5100818f5900030136007fb09700d5
:100ed4007400b9006010b00068007800cf80de00b4
:100ee400c0bf9f00d1bf9f007fb097007400b900be
:100ef4002011b000e80178004fba9700dfba9700dc
:100f04007fb097007400b900a010b00068007800aa
:100f1400040178008000eb00030001007fb097001b
:100f24007400b900a010b00068007800a0509000d0
:100f34008180fb00305090004800dd00008070008c
:100f44004fb99700dfb99700020878007fb0970087
:100f54007400b900a010b00068007800a058900098
:100f64008180fb00305890004800dd000080700054
:100f74004fb99700dfb99700020878007fb0970057
:100f84000000e800f0b79f00118680007fb0970052
:100f9400808f5000c3ff3e00500020003cff37000c
:100fa4001840a00092ff3700e8b09000181090009d
:100fb4000080500060b49800e8b0900038109000b1
:100fc400808f50004dfe3100b810900061b498003d
:100fd4006fb097004f04be000080fa0000000600c6
:100fe4004afe3700200e200008004000bb0f070017
:100ff4002000200073ff37000000eb00f0b79f00d3
:1010040058109000ffb09700808f50008dff310082
:101014007fb097007400b900a010b000e800780019
:10102400114090000074a100904098007fb0970098
:101034000000e800f0b79f00d81090007fb0970040
:10104400808f50007fff36007fb097007400b90096
:10105400a010b000e8007800114090000074a100d6
:10106400904098007fb097000000e800f0b79f0020
:10107400d81090007fb09700808f5000e4ff3e00ae
:1010840070ff37001880a00038b89000a0c090000e
:101094008180fb0030c190004811dd0002817000a6
:1010a400d808900081004100102190001120980080
:1010b40038b8900020c190000281fb00b0c09000bd
:1010c400c808dd008100710050332000808f50007b
:1010d4000afe36000000e80020bc980038b89000f2
:1010e400a8b89000102190001120980056fe3700f7
:1010f40008007800260e0700efb09700010060009a
:10110400e0b79f00281090000000e00096003a002d
:10111400b8b89000114090000074a000904098006e
:1011240051fe3700dd890a0018000000800d200000
:1011340008004000910f070080c46400dd090a0024
:1011440018000000effe3700c808900021bc98008a
:1011540038b89000a8b89000102190001120980091
:1011640068fe37000000eb00f0b79f001086800097
:10117400ffb09700808f50000eff31007fb09700c2
:101184007400b900a010b000e8007800114090008d
:101194000074a100904098007fb097007400b900db
:1011a400e010b000e80078007fb197007411b90036
:1011b400a010200002004000680078000100010037
:1011c4007fb097007400b900a010b00068007800e8
:1011d400205190000281fb00b0509000c808dd004f
:1011e400810071007fb197007411b900a010200034
:1011f400020040006800780000c190000281fb00fa
:1012040010c090004800dd00820870007fb0970095
:101214000000e800f0b79f00118680007fb09700bf
:10122400808f5000e3fe36007fb097007400b90051
:10123400a010b000e8007800114090000074a100f4
:10124400904098007fb097007400b900e010b0009f
:10125400e80078007fb197007411b900a010200055
:101264000200400068007800010001007fb0970090
:101274007400b900a010b0006800780020519000fc
:101284000281fb00b0509000c808dd0081007100ad
:101294007fb197007411b900a01020000200400033
:1012a4006800780000c190000281fb0010c090002b
:1012b4004800dd00820870007fb097000000e8005d
:1012c400f0b79f00118680007fb09700808f500098
:1012d400aaff3e00b7fe37007fb097007400b90044
:1012e4008010b000680178004fb89700dfb897000d
:1012f4008001eb00800f5100818f5900fafe31000c
:101304007fb097007400b9008010b00068007800c6
:101314008000eb00c0bf9f00d1bf9f00f2fe3700ea
:1013240028b990004fb89700dfb897008001eb0010
:10133400800f5100818f59003bfe310028b8900086
:101344008000eb00c0bf9f00d1bf9f0036fe370076
:101354001880a1006fb097004f04be000080fa000f
:101364000000060069fd370028109000e20f5000cd
:10137400bdfd3a00b8b89000114090000074a00080
:10138400904098000000eb00f0b79f00d810900048
:101394007fb09700808f5000b3fd36007fb0970078
:1013a4007400b900a010b000e8007800114090006b
:1013b4000074a000904098007fb097000000e800ff
:0413c400f1ff3700fe
:020000040000fa
:1013c800f6874700889fbe008a9fbe008c9fbe009c
:1013d8008e1f780010002000f0af9f006a182100cf
:1013e8000000eb00000d780051c22000218c88001d
:1013f80064074500a1cc2f00010f7800e6064500e0
:1014080061332000810e7800408c88006804450014
:10141800001c2100000c78008880e800627621001a
:1014280082087800a2c32100a28c880022ca210069
:10143800928c8800a2cb2100b28c880091007800a1
:10144800010001001800780041c12000f90f2000b8
:101458002041900021409800c808de0030419000eb
:1014680031409800180078009a00780040019000f8
:101478004100980018007800c0409000f0400a0031
:10148800010300004140980018007800e0409000f7
:1014980011cab30061409800f0409000c1c4b30085
:1014a8007140980018007800a0489000f0400a00a9
:1014b8000100000021489800180078008050900032
:1014c800f0400a0001000000015098001800780060
:1014d800c0489000f0400a0001050000414898000b
:1014e80018007800e048900081c5b3006148980072
:1014f800f0489000e1c5b3007148980018007800e2
:10150800ea004400098260002051900024509800ad
:10151800c809de0030519000335098001800780058
:1015280000599000f0400a0002000000025898009c
:101538001800780040519000f0400a0002000000b6
:1015480042509800180078006051900080c5eb0068
:101558006b50980070519000fac7b3007a50980009
:10156800180078007e06440009016600a2b79f00b3
:1015780020599000cfe39700275898004861de0073
:1015880092b79f0030599000afe397003758980002
:101598001800780000619000f0400a000200000086
:1015a800026098001800780040599000f0400a0046
:1015b8000200000042589800180078006059900016
:1015c8006b589800705990007a5898001800780065
:1015d80002f32f0008014100890261002063900096
:1015e800256098004811de00b062900032609800d3
:1015f800180078001e0178008022900002209800d0
:10160800180078001d0178009022900012209800a0
:101618001800780040c19000f0400a000200000065
:1016280042c098001800780060c19000f0400a009d
:101638000200000062c098001800780000c99000fd
:10164800f0400a000200000002c898001800780064
:1016580020c99000f0400a000200000022c898004b
:101668001800780040c99000f0400a00020000000d
:1016780042c898001800780060c99000f0400a003d
:101688000200000062c8980018007800e2f32f00fa
:10169800080141008902610000d3900005d098003c
:1016a8004811de0090d2900012d0980018007800ff
:1016b80040d19000f0400a000200000042d098009b
:1016c8001800780060d19000f0400a000200000085
:1016d80062d098001800780000d99000f0400a0005
:1016e8000200000002d898001800780020d9900065
:1016f800f0400a000200000022d898001800780084
:1017080040e19000f0400a000200000042e098002a
:101718001800780060e19000f0400a000200000024
:1017280062e098001800780000e99000f0400a0094
:101738000200000002e898001800780020e99000f4
:10174800f0400a000200000022e898001801780022
:10175800124090000074a100104198001801780010
:10176800124090000054a100104198001801780020
:10177800124090000044a100104198001801780020
:10178800124090000064a1001041980018007800f1
:101798001004a100180078001014a10018017800a6
:1017a800124090000034a10010419800ec0244005f
:1017b8000d8020008d0a7800e00320008008780062
:1017c800700144000705200007097800f200440072
:1017d800002c210080087800720747000769200064
:1017e800070f780074044400c0222100000c780020
:1017f80064834000e7a52100070b7800a71a2200a0
:10180800478d8800c7212200378d88004723220092
:10181800578d880016037800f1b79f00e2b79f0044
:10182800c3b79f00b4b79f00d5b79f00060001005b
:1018380018007800c6c020008903630087bf9f0096
:10184800a04390008ff39700274098004833de00ac
:10185800b04390003640980018007800dfb2970037
:101868009502780040039000450098001800780021
:10187800c0429000f0400a0005040000454098006e
:1018880018007800e04290006b409800f042900009
:101898007a40980018007800a04a9000f0400a00aa
:1018a8000500000025489800180078008052900034
:1018b800f0400a0005000000055098001800780064
:1018c800c04a9000f0400a00050000004548980012
:1018d80018007800e04a9000f0400a000500000077
:1018e8006548980018007800453820000983620090
:1018f800a053900026509800c82ade00305390006c
:101908003550980018007800805a9000f0400a007e
:10191800050000000558980018007800c052900093
:10192800f0400a00050000004550980018007800b3
:10193800e05290006b509800f05290007a50980056
:1019480018007800a05a9000f0400a000500000036
:10195800255898001800780080629000f0400a002e
:10196800050000000560980018007800c05a900033
:10197800f0400a000500000045589800180078005b
:10198800e05a90006b589800f05a90007a589800e6
:1019980018007800a06290003fb297002460980079
:1019a80030629000cfb1970033609800180078003b
:1019b8006fb19700120178008021900002209800f2
:1019c80018007800ffb0970091007800102190006f
:1019d8001120980018007800c0c09000f0400a005c
:1019e8000100000041c0980018007800e0c0900095
:1019f800f0400a000100000061c09800180078005b
:101a0800a13820000981600080c9900002c89800b0
:101a1800c808de0010c9900011c8980018007800a6
:101a28009e007800502190005120980018007800fe
:101a380021f22f00888040000981600080d1900049
:101a480002d09800c808de0010d1900011d098008c
:101a580018007800c0d09000f0400a000100000093
:101a680041d0980018007800e0d09000f0400a00bb
:101a78000100000061d098001800780080d890001c
:101a8800f0400a000100000001d898001800780012
:101a9800a0d89000f0400a000100000021d898006a
:101aa80018007800c0e09000f0400a000100000033
:101ab80041e0980018007800e0e09000f0400a004b
:101ac8000100000061e098001800780080e89000ac
:101ad800f0400a000100000001e8980018007800b2
:101ae800a0e89000f0400a000100000021e89800fa
:101af80098007800114090000074a1009040980070
:101b080098007800114090000054a100904098007f
:101b180098007800114090000044a100904098007f
:101b280098007800114090000064a100904098004f
:101b3800180078001004a100180078001014a10003
:101b480098007800114090000034a100904098005f
:101b5800720747000d0f7800e0032000000e7800a0
:101b6800f00044000205200082087800f2064400d4
:101b7800072c2100870e78006406460000692000c3
:101b8800000e78007404440080292100000c7800bd
:101b980066814000c3b42100030978004325220070
:101ba800e38d8800632c2200d38d8800e32d22006a
:101bb800f38d880012017800f1b79f000200010040
:101bc80018007800e2c020008901610020429000de
:101bd800234098004811de00b04190003240980040
:101be800180078001e017800c0019000420098009b
:101bf8001800780040419000f0400a0002040000fc
:101c08004240980018007800604190006b409800ae
:101c1800704190007a4098001800780020499000a0
:101c2800f0400a00020000002248980018007800de
:101c380000519000f0400a00020000000250980095
:101c48001800780040499000f0400a0002000000a7
:101c5800424898001800780060499000f0400a0057
:101c6800020000006248980018007800023f200037
:101c78008901610020529000235098004811de002d
:101c8800b051900032509800180078000059900028
:101c9800f0400a000200000002589800180078007e
:101ca80040519000f0400a000200000042509800a5
:101cb80018007800605190006b50980070519000a7
:101cc8007a5098001800780020599000f0400a00d7
:101cd8000200000022589800180078000061900067
:101ce800f0400a0002000000026098001800780026
:101cf80040599000f0400a00020000004258980045
:101d080018007800605990006b589800705990003e
:101d18007a58980018007800206190004fe19700e9
:101d28002260980030619000afe397003760980018
:101d380018007800ffb0970091007800002190000b
:101d480001209800180078009d007800102190006c
:101d58001120980018007800c0c09000f0400a00d8
:101d68000100000041c0980018007800e0c0900011
:101d7800f0400a000100000061c0980018007800d7
:101d8800613f20000981600080c9900002c8980066
:101d9800c808de0010c9900011c898001800780023
:101da8009c0078005021900051209800180078007d
:101db80001f12f00888040008984600000d19000e4
:101dc80009d09800c808de0010d1900011d0980002
:101dd80018007800c0d09000f0400a000100000010
:101de80041d0980018007800e0d09000f0400a0038
:101df8000100000061d098001800780080d8900099
:101e0800f0400a000100000001d89800180078008e
:101e1800a0d89000f0400a000100000021d89800e6
:101e280018007800c0e09000f0400a0001000000af
:101e380041e0980018007800e0e09000f0400a00c7
:101e48000100000061e098001800780080e8900028
:101e5800f0400a000100000001e89800180078002e
:101e6800a0e89000f0400a000100000021e8980076
:101e780098007800114090000074a10090409800ec
:101e880098007800114090000054a10090409800fc
:101e980098007800114090000044a10090409800fc
:101ea80098007800114090000064a10090409800cc
:101eb800180078001004a100180078001014a10080
:101ec80098007800114090000034a10090409800dc
:101ed8007fa897004f0778004f06be004f05be0049
:0c1ee8004f04be006f01b10000000600b6
:020000040000fa
:101ef4000800fa00889fbe008a9fbe0011002000df
:101f040081bf9f008000eb0091bf9f0091bf9f00a5
:101f1400501190009fb89700810f510020013600a6
:101f2400a532200007362000858353008783d10023
:101f3400c6e1200004e020001fb997007e11b9001b
:101f4400c109200082804000e0807800a1bf9f008a
:101f54001fb997007e11b900e1092000828040007a
:101f6400e0807800b1bf9f00bfb897000401530020
:101f74000191b90002014200afb897008100d0007e
:101f84008180e900078cb90088804200e24190001a
:101f94008381fb00f2449000c84cdd008984710009
:101fa4001fbd97007e55b900030a20008a814100b5
:101fb4006084790013002000081cdd000884ea0016
:101fc40009046400b204900038019800624590004e
:101fd4000a85fb00f2449000c84cdd0089047500ba
:101fe4001fbd97007e55b900280a20000a0444004a
:101ff40060047c00081cdd000884ea000904640015
:10200400b204900038019800224590000a85fb0034
:10201400b2449000c84cdd00890475001fbd9700d0
:102024007e55b900080a20000a04440060047c00bc
:10203400081cdd000884ea0009046400920490008e
:1020440018019800224590000a85fb00b2449000d4
:10205400c84cdd00890475001fbd97007e55b9008a
:10206400280a20000a04440060047c00081cdd00e7
:102074000884ea000904640092049000180198009e
:10208400424d90000a85fb00d24c9000c84cdd0004
:10209400890475001fbd97007e55b900080a200009
:1020a4000a04440060047c00081cdd0008847400f9
:1020b400e204900068019800424d90000a85fb00fc
:1020c400d24c9000c84cdd00890475001fbd9700f8
:1020d4007e55b900280a20000a04440060047c00ec
:1020e400081cdd0008847400e20490006801980074
:1020f400f0400a0011880000214190000041eb00eb
:10210400a240980031449000b3409800614490008c
:10211400e24098007141900002c3b300f24098007d
:1021240001499000f0400a00020000008248980033
:102134002149900092c1b300a2489800314990000f
:1021440092c0b300b24898004149900002c4b30061
:10215400c248980051499000d348980021519000fa
:10216400f0400a0002000000a25098004151900083
:10217400f0400a0002000000c2509800614990003b
:10218400f0400a0002000000e2489800015190006b
:10219400f0400a0002000000825098006151900053
:1021a400f0400a0002000000e2509800015990003b
:1021b400f0400a0002000000825898002159900063
:1021c400f0400a0002000000a25898004159900013
:1021d400f0400a0002000000c258980061599000c3
:1021e400f0400a0002000000e258980001619000eb
:1021f400f0400a0002080000826098001fb99700ae
:102204007e14b900420a20000801410060447900ac
:1022140061446400620020000244dd00314190000a
:102224000264a10008417100b2409800216190004d
:10223400f0400a0002000000a26098001fb9970055
:102244007e14b900c20a200008014100600179002f
:1022540021149000a210980061619000f0400a00df
:1022640002000000e26098001fb997007e14b900d4
:10227400620a2000080141006001790041149000c5
:10228400c210980021699000f0400a00020000008a
:10229400a268980041699000f0400a000200000022
:1022a400c268980061699000f0400a0002000000d2
:1022b400e26898001fb997007e14b900220b200031
:1022c4000801410060017900011c90008218980007
:1022d4001fb997007e14b900020b200008014100c9
:1022e40060017900111c9000921898001fb99700a2
:1022f4007e14b900420b20000801410060017900fe
:10230400710c9000f208980001619000f0400a00fe
:1023140002080000826098001fb997000200e000e4
:1023240024003a00314190000234a000b2409800e9
:102334003141900020030a0002000000b2409800de
:102344002141900030400a0002000000a2409800a1
:102354002149900020400a0002030000a24898008e
:102364001fb997007e11b900820ab000600179009c
:10237400f1119000f2109800414190000234a00045
:10238400c24098009fb897008100e80091bf9f0069
:10239400501190009fb89700810f5100e6fe3e0057
:1023a4000fb897004f05be004f04be000080fa002e
:1023b40000000600314190000234a100b2409800b0
:1023c4003141900020400a0002030000b24098000e
:1023d4002141900030400a0002020000a24098000f
:1023e4002149900020400a0002000000a248980001
:1023f4001fb997007e11b900820ab000600179000c
:10240400f1119000f2109800414190000234a000b4
:10241400c24098009fb897008100e80091bf9f00d8
:10242400501190009fb89700810f5100c2fe3e00ea
:04243400dbff370093
:020000040000fa
:102438000600fa00889fbe008a1f7800100020005e
:10244800b0bf9f008000eb00c1bf9f000040eb00c1
:10245800c0f79f00c08480000010a100c0848800dd
:10246800c08480000020a100c0848800c08480004f
:102478000030a100c0848800c08480000040a10012
:10248800c0848800c08480000070a000c0848800d8
:10249800c08480000090a000c0848800c0848000b0
:1024a80000e0a000c0848800c084800000f0a10083
:1024b800c0848800a00921000008eb00200020004b
:1024c800e0858800e20320000286880052c22000ce
:1024d800f285880010868800c1bf9f0011868000a1
:1024e8004fb89700808f500009003600420c210039
:1024f8000009eb004fb897000000e800c0bf9f003c
:10250800118680004fb89700808f5000f8ff3e007a
:10251800800c21000008eb00640040000008eb007c
:102528000080e9000008eb00640040000008eb00b0
:1025380026002000a689880010002000b0898800a5
:10254800c1002000c1898800d1002000d1898800fd
:10255800c11321008048780009f42100f989880016
:1025680008fa2000088a880002052000228a8800cc
:10257800128a8800072c2100378a880081022000ef
:10258800418a8800518a8800051e2000658a8800d3
:10259800031521008009eb008381e9008009eb0025
:1025a80043002000938a8800a08a880094002000b5
:1025b800b48a880084002000c48a8800aa152100f3
:1025c800004d7800e98a8800f88a8800128b880014
:1025d800028b8800278b8800318b8800418b88000c
:1025e800558b8800f40045008008eb00f200450098
:1025f8008008eb00838040008048eb00ea804000c0
:1026080080487800e08b8800f08b8800e6804000e6
:102618008008eb00868040008008eb00e109b100eb
:1026280080487800c0f79f00668140000349780021
:10263800678140000449780042c120003287880041
:1026480065c0b30004814000054978006b814000f3
:102658000049eb000281e900cff3970007497800b1
:1026680000014100cff3970007497800630141005a
:102678000049eb000201e9000049eb0012ca2400fe
:102688009287880032002000a2878800f2834000e9
:10269800800beb0091407800e1c360008083630009
:1026a800833bdd00017080000140a1008180730040
:1026b8000170880061f72f008a8040008048780008
:1026c800e6834000864b780067834000044b78001f
:1026d80004c1200094868800a4c0b3006883400029
:1026e800044b780002034300004beb000683e9002b
:1026f800004beb0000034300004beb0002034300d8
:10270800004beb000603e900004beb0086e52500d3
:10271800f6868800560020000687880072834000ed
:10272800000beb009140780061c360000003630078
:102738004733dd00e17080000170a1008100730063
:10274800e1708800210220008780400080487800de
:1027580066834000004beb0067834000004beb00b2
:10276800c6c02000d687880068834000054b7800e3
:10277800eb824000804aeb00e9824000804aeb008f
:1027880080824200804aeb0082824200804aeb004d
:102798008502e900804aeb00f5ff270035888800ac
:1027a800438888000380200053888800914078007f
:1027b800e1c0600000210a00000e0000ec004300a8
:1027c80080487800f201430080497800f301430013
:1027d80080497800e3c0200073888800f401430032
:1027e80084497800f70143008049eb008381e900c0
:1027f8008049eb00808141008049eb0082814100e3
:102808008049eb008301e9008049eb0091407800a2
:10281800e1c060008080600081814000017080001c
:102828000110a1008180710001708800c1f92f009a
:10283800868040008008eb00f17c2000f18488004d
:1028480021fa2f00868040008008eb008180e90093
:102858008008eb00f48040008008eb00713e200007
:10286800b1858800d2858800d18580000100e0000c
:1028780001003a00d08588008000eb00800b210021
:102888000008eb00e0858000e20f50000d003200e8
:10289800400a21000008eb00f07c20003085880009
:1028a800a00a21000008eb0050c2200040858800e3
:1028b8003fb897004f0578004f04be000080fa002b
:1028c8000000060061858800703e20007085880041
:1028d80091858800908580000000e00002003a00a1
:1028e8001000200090858800e00320008085880083
:1028f800400a21000008eb00f07c200030858800a9
:10290800a00a21000008eb0050c220004085880082
:102918003fb897004f0578004f04be000080fa00ca
:0829280000000600e7ff370084
:020000040000fa
:102930000400fa000002780011002000f1bf9f009f
:102940001404e00047003200e4409000efcf500054
:1029500048003e0054499000e44090000281fb0092
:102960008180fb008110dd0001007800d02bb700d2
:1029700024499000e44090000281fb008180fb002c
:102980008110dd0001007800f02bb70014499000a1
:10299000e44090000281fb008180fb008110dd009b
:1029a00001007800202bb700e4409000e7cf5000f2
:1029b0004f003e00e440900081c04000c1ff9f00f6
:1029c000e440900002b1200012417800c448900019
:1029d0008180fb004ff897008081fb008308dd00b9
:1029e0008140710002b120000149780002b120004d
:1029f00012417800b44990008381fb004ff89700a2
:102a00008080fb008100e8008118dd0081407100ba
:102a100002b1200001497800e44090008180fb0071
:102a200002b820000448900000f17800f4409000c3
:102a3000e1cf500056003200e1cf50005b0039007a
:102a4000e2cf50006a003200e3cf50006100320054
:102a50008af0a800344890000004e0000100320031
:102a60008cf0a800ffb89700010078000080fa0001
:102a700000000600644190008000eb00ff4f510011
:102a8000f9ff3e0054499000e44090000281fb00b1
:102a90008180fb00f08050008110dd000100780093
:102aa000d22bb70024499000e44090000281fb0043
:102ab0008180fb00f08050008110dd000100780073
:102ac000f22bb70014499000e44090000281fb0013
:102ad0008180fb00f08050008110dd000100780053
:102ae000222bb700e4409000e7cf5000b1ff360042
:102af000e4409000efcf500033003600e4409000f7
:102b0000f7cf500041003e00e4409000f0c050007c
:102b100081c04000c1ff9f00e440900002b120004e
:102b200012417800c44890008180fb004ff8970064
:102b30008081fb008308dd008140710002b120002c
:102b40000149780002b1200012417800b449900098
:102b50008381fb004ff897008080fb008100e80034
:102b60008118dd008140710002b120000149780028
:102b7000e44090008180fb0002b8200004489000ef
:102b800000f17800f4409000e1cf5000aaff3a0035
:102b90008a30a800344890000004e000b1ff320001
:102ba0008c30a800ffb89700afff37008a10a8004c
:102bb000344890000004e000aaff32008c10a80006
:102bc000ffb89700a8ff3700e4409000e8c050002d
:102bd00079ff37008a70a800344890000004e000b4
:102be000a0ff32008c70a800ffb897009eff37004e
:102bf0008a50a800344890000004e00099ff320099
:102c00008c50a800ffb8970097ff370064419000f0
:102c10008000eb00ff4f510093ff3e00e440900026
:082c2000f8c0500064ff37000a
:020000040000fa
:102c28000400fa0012002000e2bf9f008000eb00c1
:102c3800f1bf9f000000e000200032001000e0001b
:102c480021003d00100190008000eb000200e00030
:102c58001a0032009000900011017800d000900016
:102c680081006100f1bf9f00a00090000100e0001a
:102c78000700320090009000910078002001900039
:102c88009280500001f0a7008100ea00f1bf9f0088
:102c9800a8810a0010000000e38f50005b0032009a
:102ca80010003400e58f5000760032006b003500cc
:102cb800e68f50002f0032008000eb000100780002
:102cc8000080fa0000000600610098001010a100c2
:102cd8001000a100020078000080fa000000060041
:102ce800f9ff3700e18f500052003200e28f5000a8
:102cf800f1ff3a0070019000ffb89700810f510072
:102d08006a0036001010a0001018a300240032003a
:102d180010017800e10061000104e00020003a00a1
:102d2800e00090008100e8006100980060019000d8
:102d380080089000810f5100090039001000a000a0
:102d48008008900061009800b00090000100e00049
:102d5800030032003000900000000100e0bf9f0037
:102d6800efb89700010078000080fa000000060024
:102d7800d5ff370010099000ffb89700810f510068
:102d8800e0ff3e0070019000ffb89700810f5100ee
:102d9800dcff39001010a1001018a300dcff3a0076
:102da80010017800e10061000104e0001300320026
:102db8001018a30011003a00e00090008100e8001c
:102dc8006100980060019000a0089000810f5100f8
:102dd800e3ff39001000a100a008900061009800ee
:102de800c00090000100e000ddff320040009000cc
:102df80000000100e0bf9f00d9ff37008000eb0012
:102e080061009800efb89700d6ff37007001900076
:102e1800ffb89700810f5100baff3200700190008f
:102e2800ffb89700810f5100b7ff32001010a100c2
:102e3800d9ff370070019000ffb89700810f51004b
:102e4800b0ff390010099000ffb89700810f5100ba
:102e5800adff36001010a100cfff370070019000c1
:102e6800ffb89700810f5100a6ff3a00700190004b
:102e7800ffb89700810f5100a3ff3a001010a1007e
:102e8800c5ff370010099000ffb89700810f510067
:102e9800c0ff310070019000ffb89700810f51000a
:102ea800bcff36001010a00097ff370010099000f3
:102eb800ffb89700810f510093ff31001010a10057
:042ec800b5ff37001b
:020000040000fa
:102ecc000200fa00881f7800000478000000eb0074
:102edc00e0bf9f00f0000a00180000006001210014
:102eec00c860900040649800c800de0058619000f3
:102efc0051649800e800400068619000616498009b
:102f0c00c808de00786190007164980061ff2200af
:102f1c0008699000016c9800c808de0018699000e0
:102f2c00116c9800a1ff220028699000216c980078
:102f3c00c808de0038699000316c9800218480004c
:102f4c0038199000311c980091808000481990002d
:102f5c00411c98003184800058199000511c980035
:102f6c008180800028199000211c9800018080002d
:102f7c006811900061149800118080007811900005
:102f8c00711498002180800008199000011c980091
:102f9c003180800018199000111c98008000eb0003
:102fac00e1bf9f00486990000281fb00d868900047
:102fbc00c808dd00810071006fb99700828f500046
:102fcc001400360083002100efb897006fb997000a
:102fdc004211dd0002814100c208dd008100400089
:102fec00b2187800a2107800efb897008100e800c2
:102ffc00e1bf9f00486990000281fb00d8689000f7
:10300c00c808dd00810071006fb99700828f5000f5
:10301c00edff3e008000eb00e1bf9f00686990006f
:10302c000281fb00f8689000c808dd008100710087
:10303c006fb99700828f500015003600233721009e
:10304c00efb897006fb997004211dd000281410083
:10305c008180e800c208dd0081004000b2187800d1
:10306c00a2107800efb897008100e800e1bf9f0044
:10307c00686990000281fb00f8689000c808dd00c8
:10308c00810071006fb99700828f5000ecff3e00f9
:10309c00001c210028020700a0808000f818900076
:1030ac00701c980040848000e8189000601c980008
:1030bc00100020004f0478000080fa000000060089
:020000040000fa
:1030cc000600fa0010002000d0bf9f000000eb00ab
:1030dc00e0bf9f00f0bf9f00816080005186880098
:1030ec0061608000218688007160800031868800d4
:1030fc00e0bf9f00118680006fb89700808f500052
:10310c000f003600820921006fb89700760040004e
:10311c0000004000e20078007fb89700008040007b
:10312c00f0bf9f006fb897000000e800e0bf9f0061
:10313c00118680006fb89700808f5000f2ff3e0020
:10314c007fb8970040868800528680000000eb0014
:10315c0081392000810f5100050036005286800015
:10316c001000200081c82000810f510022003e0079
:10317c0061006000c300dd00c08480000030a1004d
:10318c0000807000c084880023988000d098800054
:10319c0082998000319a8000030070000200700058
:1031ac0081007000e1806000c708dd00c0848000f1
:1031bc000070a10000807000c0848800800921008c
:1031cc00adf50700dfb8970001006000d0bf9f008d
:1031dc0093060700d0848000e40f500023003e00cb
:1031ec008099800000f0a100809988005fb897005a
:1031fc000080fa00000006000000eb006100600097
:10320c00c300dd00c08480000030a100008070008d
:10321c00c084880023988000d09880008299800018
:10322c00319a800003007000020070008100700071
:10323c00e1806000c708dd00c08480000070a10040
:10324c0000807000c0848800800921008af5070086
:10325c00dfb8970001006000d0bf9f007006070028
:10326c00d0848000e40f5000ddff3600708c8000ad
:10327c00a06090008180fb00306090004800dd0071
:10328c0000807000a0998800708c800090409000a5
:10329c0077810a0001000000cf08dd0080998000d2
:1032ac0000f0a10000807000809988005fb8970042
:0c32bc000080fa0000000600cfff370081
:020000040000fa
:1032c8000200fa000000eb00f0bf9f00000027009a
:1032d800840fb60021003200a109200080072000d9
:1032e8000001eb0053f820008049780081497800fc
:1032f80082497800207c8000e007b2000000a0002e
:10330800720520006104200043f8200081497800fc
:103318008249780080497800eca10a00840f0000f7
:10332800a8a00a00840f000080cf500006003200d9
:103338007fb897008000e800f1bf9f007138210036
:10334800810f5000f4ff36000000eb0071382100b7
:103358007fb99700810f51003a003e000000eb0052
:1033680050200a008c0f00001100200050210a0094
:10337800860f0000820c2000b0220a00880f00008f
:103388004000200064200a008a0f000020210a0063
:103398008a0f00008000eb0098210a008a0f0000c5
:1033a800a1092000120020008007200053f8200007
:1033b800804978008149780082497800eca10a00a8
:1033c800840f0000a8a00a00840f000080cf5000de
:1033d80022003200207c8000e007b2000000a0003c
:1033e800720520006104200043f82000814978001c
:1033f8008249780080497800eca10a00840f000017
:10340800a8a00a00840f000080cf500006003200f8
:103418007fb897000001e800f2bf9f0071382100d3
:10342800810f5000f4ff3600eca20a00840f000060
:10343800a8a10a00840f00000000eb00814f510092
:10344800020032000080fa000000060071382100f6
:103458007fb99700810f5100faff3e0084efa80062
:1034680084afab0006003a007fb897008000e80000
:10347800f1bf9f0071382100810f5000f8ff36001e
:103488000000eb0084afab00eeff32007138210082
:103498007fb99700810f5100eaff3e0033a00a0070
:1034a800840f0000610010000080fa000000060090
:0434b800e6ff3700f4
:020000040000fa
:1034bc000200fa008000eb00f1bf9f00f0010a004f
:1034cc0010000000e1032100406190004160980071
:1034dc004809de00d061900052609800688140007d
:1034ec00e0619000626098004811de00f06190008d
:1034fc0072609800c2fe22008069900002689800f9
:10350c004811de00906990001268980002ff2200ba
:10351c00a0699000226898004811de00b069900004
:10352c003268980072848000b019900032189800ac
:10353c00e2818000c01990004218980082848000bb
:10354c00d019900052189800d2818000a0199000d8
:10355c002218980052818000e011900062109800af
:10356c0062818000f01190007210980072818000ce
:10357c0080199000021898008281800090199000a8
:10358c00121898000001eb00f2bf9f00c069900078
:10359c008381fb00506990004811dd0002817100ad
:1035ac00ffb99700830f510014003600240321004b
:1035bc007fb99700ffb99700c219dd008301420063
:1035cc004211dd000281400033197800231178008c
:1035dc007fb997000201e800f2bf9f00c06990001c
:1035ec008381fb00506990004811dd00028171005d
:1035fc00ffb99700830f5100edff3e000001eb0077
:10360c00f2bf9f00e06990008381fb00706990001d
:10361c004811dd0002817100ffb99700830f510042
:10362c0015003600e43721007fb99700ffb99700e9
:10363c00c219dd00830142000281e8004211dd0065
:10364c000281400033197800231178007fb997006c
:10365c000201e800f2bf9f00e06990008381fb004b
:10366c00706990004811dd0002817100ffb997006c
:10367c00830f5100ecff3e00c02221006b030700ba
:0c368c00100020000080fa000000060082
:020000040000fa
:103698000200fa008000eb00f1bf9f00f0010a0071
:1036a8001000000061062100406190004160980010
:1036b8004809de00d061900052609800688140009f
:1036c800e0619000626098004811de00f0619000af
:1036d8007260980022fe22008069900002689800bb
:1036e8004811de00906990001268980062fe22007e
:1036f800a0699000226898004811de00b069900027
:103708003268980092848000b019900032189800ae
:1037180022838000c019900042189800a28480007b
:10372800d01990005218980012838000a0199000b8
:103738002218980092828000e01190006210980090
:10374800a2828000f011900072109800b28280006e
:103758008019900002189800c28280009019900089
:10376800121898000001eb00f2bf9f00c06990009a
:103778008381fb00506990004811dd0002817100cf
:10378800ffb99700830f510014003600a4052100eb
:103798007fb99700ffb99700c219dd008301420085
:1037a8004211dd00028140003319780023117800ae
:1037b8007fb997000201e800f2bf9f00c06990003e
:1037c8008381fb00506990004811dd00028171007f
:1037d800ffb99700830f5100edff3e000001eb0099
:1037e800f2bf9f00e06990008381fb007069900040
:1037f8004811dd0002817100ffb99700830f510065
:1038080015003600a43821007fb99700ffb997004a
:10381800c219dd00830142000281e8004211dd0087
:103828000281400033197800231178007fb997008e
:103838000201e800f2bf9f00e06990008381fb006d
:10384800706990004811dd0002817100ffb997008e
:10385800830f5100ecff3e00802921004903070037
:0c386800100020000080fa0000000600a4
:020000040000fa
:1038740010f0a6002d003700201490004015900091
:103884008608c3008608c1001201c100301b9000e5
:103894000600c8001a039000260598000a03900049
:1038a40016059800100190009200780000299000fd
:1038b40001097800101190009280100020199000e6
:1038c4008208dd0030149000010d78008688c30062
:1038d4008688c1008688c1001281c100401b900007
:1038e4000680c8000000cb000400cd001023900027
:1038f40016a0e60006027800002390001620e600d9
:1039040006027800100c9000040c7800500c900013
:10391400040c7800401590000a03900016059800e6
:10392400040d7800a01c04000000000010019000a9
:103934009200780000299000010978000000060038
:10394400801f7800401090000018eb000008eb0086
:103954004f007800801f7800501090000018eb0092
:103964000018eb000008eb004f0078000000060090
:10397400801f7800811f7800501090000118780093
:103984000118780001087800cf0078004f00780013
:10399400801f7800821f7800401090000218780081
:1039a400020878004f0178004f00780000000600fc
:1039b40010f0a6001a003700100190009200780061
:1039c40000299000010978001011900092801000e5
:1039d400201990008208dd00701b9000601990008f
:1039e400010278001301c1000200c8000400cd00e8
:1039f4001023900016a0e600060278000023900031
:103a04001620e60006027800100c9000040c7800e2
:103a1400500c9000040c78001a1d040000000000f3
:103a240010019000920078000029900001097800ac
:043a34000000060088
:020000040000fa
:103a38000200fa0011002000f1bf9f00a52fa90085
:103a48002be3a90061e3a90097e3a900cde3a9004e
:103a580031002000f0210a0000030000213020007e
:103a680091407800f0400a00010000002230200058
:103a7800014978004130200091407800f0400a0068
:103a88000100000042302000014978006130200028
:103a980091407800f0400a000100000062302000e8
:103aa800014978008130200091407800f0400a00f8
:103ab800010000008230200001497800a130200078
:103ac80091407800f0400a0001000000a230200078
:103ad80001497800c06091000104e0000300320051
:103ae8003090900051188000501888000cc3bf0017
:103af800f0400a00000000000ce3b7000ec3bf004e
:103b0800f0400a00000000000ee3b70010c3bf0039
:103b1800f0400a000000000010e3b70012c3bf0025
:103b2800f0400a000000000012e3b70014c3bf0011
:103b3800f0400a000000000014e3b70016c3bf00fd
:103b4800f0400a000000000016e3b70018c3bf00e9
:103b5800f0400a000000000018e3b7001ac3bf00d5
:103b6800f0400a00000000001ae3b7001cc3bf00c1
:103b7800f0400a00000000001ce3b7001ec3bf00ad
:103b8800f0400a00000000001ee3b70020c3bf0099
:103b9800f0400a000000000020e3b70022c3bf0085
:103ba800f0400a000000000022e3b70024c3bf0071
:103bb800f0400a000000000024e3b70026c3bf005d
:103bc800f0400a000000000026e3b70028c3bf0049
:103bd800f0400a000000000028e3b7007fb8970013
:083be8000080fa000000060055
:020000040000fa
:103bf0009610000002000000800000000413000086
:103c0000580000008000000098100000280100000b
:103c1000800000007a1000000a0000008000000010
:103c20008a100000040000008000000072130000f1
:103c30000c00000082000000c4720000006f010050
:103c40000000ac008e000000c01100006c000000fd
:103c5000800000000010000016000000820000003c
:103c60000200030000020000030072007100000067
:103c70008f0e0000000300000300d6005400000077
:103c800084100000060000008000000016100000f4
:103c90001400000080000000f62f00000a00000061
:103ca000800000007e1300000c0000008200000075
:103cb000287d000000cd0e000000a600910000004d
:103cc0002c1200006c000000800000002a10000090
:103cd0001400000082000000020003000002000047
:103ce0000300bd005800000044270000000300004e
:103cf000050000008e10000004000000800000009d
:103d00003e1000001400000080000000ec2f0000b6
:103d10000a000000800000008a1300000c00000070
:103d200082000000287d000000cd0e000000a600eb
:103d300091000000981200006c000000800000005c
:103d40005210000014000000820000000200030076
:103d5000000200000300bd005800000044270000de
:103d600000030000050000009210000004000000a5
:103d700080000000661000001400000080000000b9
:103d8000e22f00000a000000800000000000000098
:020000040000fa
:103d90000800fa0011002000c1bf9f008000eb0066
:103da000d1bf9f00e1bf9f00f1bf9f00d1bf9f0027
:103db00050119000dfb89700810f51004e0036007f
:103dc000a432200005362000848252008582d10072
:103dd0005fb997007e11b900c109200082804000c0
:103de000e0807800f1bf9f007fb997000201d0000a
:103df0000281e9000591b90082004200e141900092
:103e00008381fb00714190004811dd000281710047
:103e10000300230002817100b1019000b2009800fc
:103e2000814990008381fb00114990004811dd0019
:103e30000281710033ff2f0003016100c101900076
:103e4000c2009800114190000274a00092409800b6
:103e5000414190000234a000c24098001181fb0053
:103e6000914190000278a3000e0032000003e200ae
:103e7000060035006fb997008201e800e3bf9f009c
:103e800073382100830f5100f8ff3600efb9970017
:103e900072382100828f51001a003e0001c3ab002e
:103ea00018003a00814990008381fb00114990007d
:103eb0004811dd0002817100c200b300c101900011
:103ec000c20098009140900077810a000100000034
:103ed0004fb9970082806000c1bf9f00dfb8970094
:103ee0008100e800d1bf9f0050119000dfb897001b
:103ef000810f5100b6ff3e004fb897000080fa00d6
:103f0000000006000000eb000080fa000000060040
:043f1000fcff37007b
:020000040000fa
:103f1400889fbe00a90c2100399888008000eb001e
:103f2400419888008082eb00759888004630210013
:103f3400f48f2f00160062000090a000000b7800a0
:103f440081988800803920009098880027032000f9
:103f5400a7988800703e2000b0988800481f200071
:103f6400c89888008399220053988800629e220092
:103f740062988800a03121001010a0001000a00059
:103f840016f0a000e9988800f19888002599880027
:103f9400100362000680a0000608780031998800aa
:103fa40096c820004699880057998800e604b10015
:103fb4006699880078998800039988001299880086
:103fc4001010a0001000a00010f0a0000980e8006c
:103fd400909988006c805400a0998800d599880035
:103fe40000332100100362000680a0000608780058
:103ff400e199880016082000f6998800a60f200091
:10400400069a880096012000169a8800863e2000b1
:10401400269a8800b3998800c29988001010a100dc
:104024001000a10010f0a1000980e900409a880066
:10403400519a8800859a8800603421001002620039
:104044000480a00004087800919a8800c1662100c9
:10405400a19a8800b79a8800d105b100c19a880056
:10406400017d2000d19a8800639a8800729a8800a2
:104074001010a0001000a00010f0a00010002000fc
:084084004f04be00000006001d
:020000040000fa
:10408c000200fa0012002000f2bf9f009002900084
:10409c0003e02000c1e1200083805000058ab900b4
:1040ac0084804100b00190000300e00028003a0039
:1040bc00614290000482fb00f1419000c819dd00c0
:1040cc0083017200200290000411dd000281ea00dd
:1040dc0003016100b1019000b20098004001900012
:1040ec000200e00027003200214290000482fb0015
:1040fc00b1419000c819dd008301720020019000cd
:10410c00140020000221dd00028171009101900059
:10411c00920098001182fb0091419000c819dd00bb
:10412c008301720020019000100020000201dd00cc
:10413c000281ea0003016100f0020a001100000094
:10414c00f0bf9f007fb897000080fa0000000600c7
:10415c00614290000482fb00f1419000c819dd001f
:10416c0083017200200290000411dd0002817100b5
:10417c00b1019000b2009800400190000200e000f4
:10418c00d9ff3a00214290000482fb00b14190001b
:10419c00c819dd008301720020019000140020007a
:1041ac000221dd000281ea0003016100910190000f
:1041bc00920098001182fb0091419000c819dd001b
:1041cc008301720020019000100020000201dd002c
:1041dc000281ea0003016100f0020a0011000000f4
:1041ec00f0bf9f007fb897000080fa000000060027
:0441fc00d7ff3700b2
:020000040000fa
:104200000600fa0011002000d1bf9f008000eb00e3
:10421000e1bf9f00f1bf9f00e1bf9f0050119000e0
:10422000efb89700810f510047003600a3322000fd
:1042300004362000030252000482d100efb8970038
:104240007e0bb900c109200086804000e080780024
:10425000f1bf9f00ffb897008100d0008180e90086
:10426000048bb90086804100e14290008582fb000a
:10427000714190004811dd000281720005002300a9
:1042800002817200b1029000b2009800814a900051
:104290008582fb00114990004811dd000281720007
:1042a00035ff2f0005016100c1029000c200980097
:1042b0009182fb00114190004811dd0002817200e3
:1042c00002f0a100f0020a00110000006fb997008f
:1042d0007e13b900c20a2000060141006001790086
:1042e000a1129000a2109800c14290008582fb00ac
:1042f000514190004811dd00028172000230a0009f
:10430000a1029000a20098001141900001c8b300e2
:10431000814061008180fb008100e900cf08de0060
:104320005fb9970082806000d1bf9f00efb897000f
:104330008100e800e1bf9f0050119000efb89700a6
:10434000810f5100bdff3e005fb897000080fa006a
:044350000000060063
:020000040000fa
:1043540010f0a600320037002014900040159000a1
:104364008608c3008608c1001201c100301b9000fa
:104374000600c8001a039000260598000a0390005e
:104384001605980010019000920078000029900012
:104394000109780040019000810011001011900083
:1043a40092801000201990008208dd0030149000e3
:1043b400010d78008688c3008688c1008688c10004
:1043c4001281c100401b90000680c8000000cb0091
:1043d4000400cd001023900016a0e6000602780029
:1043e400002390001620e60006027800100c9000ce
:1043f400040c780041a3de0050249000080543001b
:10440400402490000a0c7800401590000a039000a4
:1044140016059800040d78001a220400000000001c
:1044240010019000920078000029900001097800a2
:1044340000000600801f7800401090000018eb0078
:104444000008eb004f007800801f780050109000a7
:104454000018eb000018eb000008eb004f00780098
:1044640000000600801f7800811f78005010900023
:10447400011878000118780001087800cf0078004e
:104484004f007800801f7800821f78004010900051
:1044940002187800020878004f0178004f00780075
:1044a4000000060010f0a60032003700201490002f
:1044b400401590008608c3008608c1001201c1009f
:1044c400301b90000600c8001a03900026059800cf
:1044d4000a039000160598001001900092007800dd
:1044e400002990000109780040019000810011002a
:1044f4001011900092801000201990008208dd00b5
:1045040030149000010d78008688c3008688c100ad
:104514008688c1001281c100401b90000680c8003b
:104524000000cb000400cd001023900016a0e6008c
:1045340006027800002390001620e60006027800a8
:10454400100c9000040c780041a3de00502490006d
:1045540008054300402490000a0c780040159000a0
:104564000a03900016059800040d7800c422040084
:1045740000000000100190009200780000299000d3
:104584000109780000000600801f780040109000a8
:104594000018eb000008eb004f007800801f780043
:1045a400501090000018eb000018eb000008eb001e
:1045b4004f00780000000600801f7800811f7800fb
:1045c4005010900001187800011878000108780054
:1045d400cf0078004f007800801f7800821f780099
:1045e4004010900002187800020878004f0178000b
:0845f4004f00780000000600f2
:020000040000fa
:1045fc000200fa0010002000f0bf9f00a40fa900d9
:10460c0001eba90001aba9003100200065210a00d3
:10461c00020b000002eba90005eba90005cba900d9
:10462c00058ba80071002000a8210a00040b0000d3
:10463c0060200a00040b00008100200090210a0079
:10464c00060b000007cba90007eba9008000eb00cc
:10465c00fd210a00080b0000098ba900096ba900b9
:10466c00094ba900092ba900090ba90008eba9000b
:10467c0008cba90050210a00080b0000fe200a00fc
:10468c000a0b0000d8210a000a0b00000aeba90053
:10469c000a0ba9000a2ba9000c0ba9000c2ba900d2
:1046ac0010210a000e0b000032200a000e0b000035
:1046bc0000eca900000ca900002ca900f0002000bf
:1046cc00b8200a00020c000002eca900020ca900a0
:1046dc00022ca90090210a00d80b000090210a009e
:1046ec00d40b00003100200098210a00d60b0000ea
:1046fc000000eb0060200a00d60b000071002000c7
:10470c00ca210a00d60b00003000200098200a00b5
:10471c00da0b00008000eb0060210a00da0b0000cd
:10472c0070002000ca200a00da0b00007fb8970046
:08473c000080fa0000000600f5
:020000040000fa
:104744000400fa00881f780018002000d8bf9f00da
:104754000000eb00e0bf9f00dafa0700dfb8970023
:1047640001006000d0bf9f004d020700dfb8970032
:1047740001006000d0bf9f00c1020700dfb89700ae
:1047840001006000d0bf9f0021020700dfb897003e
:1047940001006000d0bf9f0023eea800f3020700d1
:1047a400dfb8970001006000d0bf9f00cb02070074
:1047b400dfb8970001006000d0bf9f0008007800b8
:1047c400ad000700dfb8970001006000d0bf9f0074
:1047d40076020700dfb8970001006000d0bf9f0099
:1047e40042010700dfb8970001006000d0bf9f00be
:1047f400c7fd0700dfb8970001006000d0bf9f002d
:104804000000eb0064200a00400800000028a90012
:104814002028a90001e1a800000880004f00de0064
:10482400dfb8970001006000d0bf9f0023eea9000d
:104834005fb897000000e00001003a000000fe00ad
:104844000028ab0006003a006fb897008000e8002b
:10485400e1bf9f00f1522700810f5000f8ff36009e
:104864000028a9000000eb00e0bf9f0023eea80091
:1048740015fa07006802070023eea90000000000f3
:04488400efff37000b
:020000040000fa
:104888000600fa0011002000d1bf9f008000eb0055
:10489800e1bf9f00e1bf9f0050119000efb8970063
:1048a800810f510036003600a43220000536200062
:1048b800848252008582d1006fb997007e11b900b9
:1048c800c109200082804000e0807800f1bf9f008d
:1048d8007fb997000201d0000281e9000591b90073
:1048e80082004200e14190008381fb007141900009
:1048f8004811dd000281710003002300028171006c
:1049080031039000b200980041619000f0400a0025
:1049180002000000c2609800414390000683fb003b
:10492800514190004811dd00020173000230a000df
:1049380021039000a2009800614190000281fb00d1
:10494800f1409000c808dd0081007100838160009b
:104958008301ea00cf19de00dfb89700818161008a
:10496800d3bf9f00efb897008100e800e1bf9f0028
:1049780050119000efb89700810f5100ceff3e0014
:0c4988005fb897000080fa0000000600f5
:020000040000fa
:104994000600fa0011002000d1bf9f008000eb0048
:1049a400e1bf9f00f1bf9f00e1bf9f005011900045
:1049b400efb89700810f51002c003600a33220007d
:1049c40004362000030252000482d100efb897009d
:1049d4007e0bb900c109200086804000e080780089
:1049e400f1bf9f00ffb897008100d0008180e900eb
:1049f400048bb90086804100414190000234a0003c
:104a0400c2409800e14290008582fb007141900011
:104a14004811dd0002817200f5ff2c0005016100e0
:104a2400b1029000b200980061419000f140900002
:104a3400c808dd0002002300828060008100e900d4
:104a4400cf08de005fb9970082806000d1bf9f006d
:104a5400efb897008100e800e1bf9f00501190007b
:104a6400efb89700810f5100d8ff3e005fb8970060
:084a74000080fa0000000600ba
:020000040000fa
:104a7c000400fa00f0bf9f0012002000e2bf9f006c
:104a8c007fb8970081c8200084c920000102520021
:104a9c000000e90000a2b9000480400090409000a2
:104aac000174a10011409800a040900001ceb30009
:104abc0021409800b0419000c1cfb30081c061008b
:104acc000104a000314098009040900065400a001d
:104adc000100000011409800904090000124a100ba
:104aec0011409800904090000104a10011409800e2
:104afc001064a10053400a00100000001024a10013
:104b0c0010400a0010000000904090000114a0001a
:104b1c0011409800e040900080c0eb00614098008c
:104b2c00f040900071c0b300714098007fb89700be
:104b3c000000e9000011dd00b28488006fb8970016
:084b4c000080fa0000000600e1
:020000040000fa
:104b54000200fa00881f780018002000e8bf9f00b8
:104b640080092100b3fb0700efb897000100600043
:104b7400e0bf9f0080092100ddf40700efb8970033
:104b840001006000e0bf9f009bfe0700efb89700a4
:104b940001006000e0bf9f00400e210063f70700a2
:104ba400efb8970001006000e0bf9f00000d2100f6
:104bb4005ef70700efb8970001006000e0bf9f00b8
:104bc400800f210059f70700efb89700010060003b
:104bd400e0bf9f00c010210054f70700efb8970012
:104be40001006000e0bf9f00001221004ff70700a2
:104bf400efb8970001006000e0bf9f00800921002a
:104c04004a010700efb8970001006000e0bf9f0071
:104c140032280a000e0b00006fb897004f0478008a
:084c24000080fa000000060008
:020000040000fa
:104c2c00d0848000e20f500001003200000006002a
:104c3c00c08480000048a300fcff3a00c0848000c0
:104c4c000018a300f9ff32007a30ec00d08380000a
:104c5c00e70f50001a003600e083800021868000a8
:104c6c0000804000e0838800008480003186800052
:104c7c000080400000848800e08380004300de0058
:104c8c00e0838800008480004300de0000848800fc
:104c9c00108d8000e183800040019000410098005d
:104cac00b08d80000184800040019000410098008c
:104cbc00c08480000040a000c08488000000060072
:104ccc00e08380002186800000804000e083880023
:104cdc0000848000318680000080400000848800c1
:044cec0000000600be
:020000040000fa
:104cf0000200fa0010002000f0bf9f00cef5070070
:104d0000ffb8970001006000f0bf9f00aef1070000
:104d1000ffb8970001006000f0bf9f008dff070003
:104d2000ffb8970001006000f0bf9f0080092100dc
:104d300017fc0700ffb8970001006000f0bf9f005c
:104d40007fb897000000e00003003200c0848000bc
:104d50000020a000c08488000f000700ffb8970063
:104d600001006000f0bf9f00f00ba8005000200081
:104d7000ec200a006c0800000b68a9002b68a80052
:104d8000c084800000f0a000c08488007fb8970035
:084d90000080fa00000006009b
:020000040000fa
:104d98000600fa0010002000d0bf9f000000eb00c2
:104da800e0bf9f00f0bf9f0001eba8008a10f80049
:104db800000cf900508480004800dd008a10b7001c
:104dc800f0bf9f00036080007fb997006fb897001d
:104dd8008000e800e1bf9f0071382100810f50007a
:104de8000a0036006fb997000000eb007138210007
:104df800810f510003003e008a10f8000a0bf900e9
:104e08005fb897000080fa0000000600828f51000a
:104e1800f4ff3200036080007fb997006fb89700f5
:104e28008000e800e1bf9f0071382100810f500029
:084e3800ecff3e00f5ff37001e
:020000040000fa
:104e40000200fa0012002000f2bf9f0090029000c2
:104e500003e02000c1e1200083805000058ab900f2
:104e600084804100b00190000300e0000e00320099
:104e7000614290000482fb00f1419000c819dd00fe
:104e800083017200200090000011dd000281ea0021
:104e90000301610031009000b20098007fb89700d4
:104ea0000080fa0000000600614290000482fb00ce
:104eb000f1419000c819dd008301720020009000cc
:104ec0000011dd000281710031009000b2009800f5
:104ed0007fb897000080fa0000000600f2ff37005c
:020000040000fa
:104ee0000200fa0012002000f2bf9f009002900022
:104ef00003e02000c1e1200083805000058ab90052
:104f000084804100b00190000300e0000d003200f9
:104f1000614290000482fb00f1419000c819dd005d
:104f200083017200200090000011dd0002817100f9
:104f300031009000b20098007fb897000080fa001e
:104f400000000600614290000482fb00f1419000e5
:104f5000c819dd0083017200200090000011dd00ff
:104f60000281ea000301610031009000b200980064
:104f70007fb897000080fa0000000600f1ff3700bc
:020000040000fa
:104f80000200fa0011c0b300e1ff9f009001900001
:104f900001e02000c2e12000010151000391b900ad
:104fa00002814000c24190008381fb005241900089
:104fb0004811dd0002817100a00090001300200064
:104fc0008118dd008280600001f0a7008100ea0006
:104fd0008100ea00cf08de00e1ff9f003000900072
:104fe000830f5000030032006ff897000080fa0032
:104ff00000000600eff897000180fb0000805100e0
:10500000e0ff9f006ff897000080fa0000000600a4
:04501000f8ff37006e
:020000040000fa
:105014000200fa0010002000f0bf9f00002eef00f5
:105024001c2eef0023cea9001fcea90023eea90059
:105034001feea900234ea9001f4ea900230ea900ac
:105044001f0ea900232ea9001f2ea9000000eb00ab
:1050540051052000b1468800a10a2000b14688000d
:105064000068880020022000d8200a00880d000073
:105074003102200050210a00880d00000080200029
:1050840051052000b1468800a10a2000b1468800dd
:10509400006888007fb897000080fa0000000600ce
:020000040000fa
:1050a4000200fa000000eb00f0bf9f008fefa900a0
:1050b4003100200098210a00920f00001000200007
:1050c40050200a008e0f0000d1072000b0210a00f2
:1050d400900f00002000200064200a00920f0000be
:1050e4001100200020210a00920f00008f0fa80059
:1050f4008fefa8000000eb008e0fe20009003d00d6
:105104008fcfab0006003a007fb897008000e8001c
:10511400f1bf9f0071382100810f5000f8ff360065
:0c512400100020000080fa0000000600cf
:020000040000fa
:105130000200fa00881f78000004780010002000a8
:10514000e0bf9f0008d891000004e00010003a0082
:1051500028e091000004e00004003a006fb89700d6
:105160004f0478000080fa0000000600200e2000a6
:1051700008004000c5fb0700e0bf9f006fb8970024
:105180004f0478000080fa0000000600f7ff3700a7
:10519000800d200008004000bcfb0700e0bf9f001e
:1051a00028e091000004e000ecff3200efff370040
:020000040000fa
:1051b0000200fa0010002000f0bf9f00b1848000c0
:1051c000cf08dd004064800000f0a1000080700086
:1051d0004064880011a10a0096100000cf08dd008d
:1051e000c064800000f0a10000807000c0648800ee
:1051f00022a10a0096100000cf08dd004065800063
:1052000000f0a100008070004065880081eca800db
:0c5210007fb897000080fa000000060044
:020000040000fa
:10521c000200fa0010002000f0bf9f004030210077
:10522c007ef60700ffb8970001006000f0bf9f00fa
:10523c00a031210079f60700ffb89700010060004b
:10524c00f0bf9f000033210074f60700ffb89700f1
:10525c0001006000f0bf9f00603421006ff6070072
:10526c00ffb8970001006000f0bf9f007fb8970067
:08527c000080fa0000000600aa
:020000040000fa
:1052840001e1a90001a1a9000181a9000161a9000e
:105294000141a9003000200098200a00000100000c
:1052a40000e1a9000000eb0054200a000001000006
:1052b4000041a9000021a9000421ef00f0702200a0
:1052c400400888000000eb0064200a004008000049
:0c52d4000028a9002028a90010000500f7
:020000040000fa
:1052e0000200fa0010002000f0bf9f0081eca9002e
:1052f00081aca9002100200076210a00800c00006a
:1053000054200a00800c00008000eb0020210a00dd
:10531000800c000090200a00840c000090200a00fd
:10532000860c00007fb897000080fa00000006009d
:020000040000fa
:105330000200fa00881f780018002000e8bf9f00d4
:105340008009210050fd0700efb8970001006000c0
:10535000e0bf9f00800921001070a000d884880061
:105360006fb897004f0478000080fa000000060034
:020000040000fa
:105370000200fa0010002000f0bf9f00dde8a90045
:10538000dc08a900dc28a800de08a800de28a800a8
:10539000de48a800dde8a8007fb897000080fa008a
:0453a0000000060003
:020000040000fa
:1053a400009b8800203621001008e800000000005f
:1053b40000000000000000000000000000000000e9
:0853c4000000000000000600db
:020000040000fa
:1053cc000200fa000000eb00f0bf9f00100020006c
:1053dc00d08488008009210010f0a0007fb89700cd
:0853ec000080fa000000060039
:020000040000fa
:04be0000ffff000040
:020000040000fa
:04be2000ffffff0021
:020000040000fa
:04be30007fffff0091
:020000040000fa
:04be38007be7ff00a5
:020000040000fa
:04be4000677fff0019
:020000040000fa
:04be4800ffffff00f9
:020000040000fa
:04be5000ddffff0013
:020000040000fa
:04be58000000ff00e7
:020000040000fa
:04be60000000ff00df
:020000040000fa
:04be68000000ff00d7
:020000040000fa
:04be70000000ff00cf
:020000040000fa
:04be7800ffffff00c9
:020000040000fa
:04be8000fffcff00c4
:020000040000fa
:04be8800c9ffff00ef
:00000001FF
